:1000000000308A00192800002230840000080319FB
:1000100018280130F800F701F70B0C28F80B0B2813
:100020004A30F700F70B122800000000800B092867
:10003000003484011F30830507309F00831685013B
:10004000FF308600831285018316811300308312EE
:10005000061A0130003A03195D280030861A013073
:10006000003A03194D280030061B0130003A0319ED
:100070003D28850183162628831205140430A1002B
:10008000FA30A2000420A10B402805100430A10082
:10009000FA30A2000420A10B482885140430A100E6
:1000A000FA30A2000420A10B502885100430A100D2
:1000B000FA30A2000420A10B582805150430A10035
:1000C000FA30A2000420A10B602805110430A10021
:1000D000FA30A2000420A10B6828831626286300AA
:02400E00693F08
:00000001FF
